:100000000C942A000C9447000C9447000C94470071
:100010000C9447000C9447000C9447000C94470044
:100020000C9447000C9447000C9447000C94470034
:100030000C9447000C9447000C9447000C94470024
:100040000C9447000C9447000C9447000C94470014
:100050000C94470011241FBECFE5D4E0DEBFCDBF16
:1000600010E0A0E6B0E0E6E1F2E002C005900D92FB
:10007000AE36B107D9F710E0AEE6B0E001C01D9290
:10008000AE36B107E1F70E94F3000C940A010C941C
:100090000000959A85E08A95F1F7959808951F9349
:1000A000182F949882B3807F82BB92B3812F829560
:1000B0008F70892B82BB0E94490082B3807F82BBF4
:1000C00082B31F70812B82BB0E94490080EE8A950B
:1000D000F1F71F9108951F93182F949A82B3807F90
:1000E00082BB92B3812F82958F70892B82BB0E9435
:1000F000490082B3807F82BB82B31F70812B82BB99
:100100000E94490080EE8A95F1F71F91089581E0E1
:100110000E944F0080E29EE40197F1F708950F934B
:100120001F9381B38F6381BB80E69AEE0197F1F74D
:1001300082B3807F82BB82B3836082BB94980E942B
:10014000490080E29EE40197F1F70E94490000EA2D
:100150001FE0C8010197F1F70E944900C80101970B
:10016000F1F782B3807F82BB919A0E944900C80157
:100170000197F1F788E20E944F008CE00E944F0047
:1001800086E00E944F000E9487001F910F91089502
:1001900082E00E944F0080E29EE40197F1F708950B
:1001A000623061F0633018F4613069F405C0633087
:1001B00039F0643041F406C0805805C0805403C053
:1001C000805701C080530E944F000895CF93DF9362
:1001D000EC0103C00E946B00219688818823D1F72F
:1001E000DF91CF9108950E948F0084E50E946B00FB
:1001F00085E60E946B0083E70E946B0084E70E9403
:100200006B0062E080E00E94D00080E690E00E94F7
:06021000E600FFCFFFCF66
:0E02160048656C6C6F20576F726C642100009D
:00000001FF
